:020000020000FC
:1000000009C02EC12DC1DCC02BC12AC129C128C104
:1000100027C1F6C00FE90DBF05E007BB06E008BB2E
:100020000FE706BF0093690022243324442455249B
:1000300066247724002700936700009365000093EF
:1000400068000093660002BF02E009BF03BF0BE82F
:1000500006B99CD0A9D0789404D018D03CD081D0D7
:10006000FBCFB19B01C00895A4D0B19BFDCF0091FF
:100070006800003029F0002700936800C0980895B8
:1000800093D001E000936800C09A08950091680041
:100090000030E9F00091670010916500011B99F0B4
:1000A00000916700011B30F0009167000550101BA4
:1000B00050F407C0009167001550011B20F4C2984E
:1000C0000895C29A0895062D0450C8F3FACF062D5C
:1000D0000030A9F3F6CF009160000132A1F4009145
:1000E00063001091640037D00093670000916500B1
:1000F0000093660000916100109162002CD0009383
:10010000650002D043D0089500916500109166000B
:10011000011B01F10091650010916600011B80F048
:100120000091650010916600101B08F013C000914B
:10013000650010916600011B8894055050F40895E5
:100140000091650010916600101B8894155008F40A
:1001500008952AD0089526E0169507952A95E1F787
:10016000089500916800003059F0009167001091E7
:100170006500011B49F0009167001250011B10F04F
:10018000C0980895C09A0895C098089503E407B9E7
:1001900000270093600000936100009362000093C9
:1001A0006300009364000895222433240BE1402E61
:1001B000089554E144274A95F1F75A95E1F70895D7
:1001C0000F939FB700916800003069F02A94022DC8
:1001D000003049F43A94032D003029F44A94042D58
:1001E000003009F448DF5A94052D003029F4639457
:1001F000062D083009F46624369A9FBF0F91189592
:100200000F931F932F933F939FB724B135B1009164
:1002100060000132F9F00395009360000131C1F0F4
:10022000015158F00091630010916400020F131FF8
:1002300000936300109364000DC000916100109161
:100240006200020F131F009361001093620002C04E
:1002500002E407B99FBF3F912F911F910F9118950D
:020260001895EF
:00000001FF
